:020000020000FC
:0200000006C038
:020004001DC01D
:10000C003FC00FE90DBF0FE007BB00E108BB02E0EA
:10001C000FBD03E003BF0FEF06BF04E009BF00E212
:10002C000BBF00E105BB00E305BF00E808B97894FD
:10003C008895FECF26B3209524FD02C000E002BFB8
:10004C0024FF0EC002B7043058F0003418F00BD067
:10005C00542F432F330F739502B7003108F03395AB
:10006C0000E205BF18953F70753039F4431719F449
:10007C00531709F40FD0772708953327772708955E
:10008C00F2DF30E041E052E060E000E002BF00E36C
:10009C0005BF18956030F9F408B33F70333039F070
:1000AC00363051F0393069F03C3081F014C000FD2D
:1000BC00C09800FFC09A0FC001FDC19801FFC19A02
:1000CC000AC002FDC29802FFC29A05C003FDC39884
:0A00DC0003FFC39A00C061E008951D
:00000001FF
